:100000001D2265007F3E62000930A0008C010C08B3
:100010002222E7218C0AA00B07289030E7210A084A
:100020000839E721F0308A051B308400840A052254
:100030008000841E162820301D0603198F282130C9
:100040001D060319A7288A0A0C30AF002F08693E45
:1000500056231D0603193028AF0B26280D28000053
:100060002F08073C031C38281D08A008031DE721A2
:100070002F083B3E8A0182005428282A5E280A293C
:10008000AB294B28B5284D287429492849286E30BA
:100090000E286B300E280630292AAC30E7211E08C6
:1000A000AE0003171E1A8A15A003A01B0D280522F7
:1000B0002A1F54289E0803198A15542883138A1569
:1000C000031F6E282E08E421200303198A1103134D
:1000D0002E08A73A0319D92970202A2A83176828DD
:1000E000A13A03193C34A23A03195F34013A0319C7
:1000F00065340D3A03194034023A03194734063A7D
:1001000003194E34013A03195534493A03195F343F
:10011000EC3A03193E34AE3A03195A340034203015
:10012000E72120088D0020308400840A0522800009
:10013000A00B95281E088A071F086323203084001F
:10014000840A00086E238D0BA0288D230D282130F2
:10015000E7212008A0001E088A001F085623E72177
:100160005C23A00BAF288D230D2820088D000D10D7
:100170008D03A00305228D0BB928EF3E8D00031CD3
:10018000A629A00305228900091A8D15891A8D1741
:100190000F398E0003198B162018052213088100D1
:1001A000D52107300E02031CEA280319F5280E1C7E
:1001B000DD280B16E4208F002F29E4202F0A562378
:1001C0008D008D142F0AF1280D080D070D07783EBC
:1001D000AF00080005089F0039212E080E078B1E6E
:1001E0000D2863230D0869232F290D08AA3A031946
:1001F00002296B300D186A308D000A3063230D0818
:10020000692363003921D5212F0A56238D000D144F
:100210002F0AF128D5219E1829291E1911298C0190
:100220000D280108A4000522A1000522A2000F3913
:1002300081000522F039A3008106210A031D0B1A53
:100240000D2839212F088B3E8C0024088A19810043
:100250000D2803308C0731210C08333C03198A1513
:100260000D288C0A8C0AD02188183129FD308C0782
:100270000800AD01AE017830AF00D5210A128A1115
:100280002F0856230F39AC005C2308180A1688186B
:100290004E29F0392C060106031959293830AE07CA
:1002A0000318AD0A0330AF07BD302F02031D3E29EE
:1002B0008A152D088A078A0A9F1107309F039F1B02
:1002C0000800AE0703188A0A5C29213084002E0832
:1002D00063235C238000840A841D69290800A0022E
:1002E0000422A00B702908000B1E80290B12D521B7
:1002F0000F03632321086E2322086E23230869233A
:100300001F088500392165212F088B3E8C00DB21D9
:100310000A3EAE005623AD002E0863230508F63EC4
:100320000318073E3A3E963AAF002F0EAD06031D66
:1003300069231A306F2165220830890014303D226C
:10034000652203228830E7210830A0000522A00B97
:10035000A6298A110D28201C2019C1293130201E00
:10036000292AA019C129EA30E4211030E4210C30F7
:1003700084000008E721840AA00BB9290108930032
:100380000D28D5210C080319AE29D021E421D02154
:10039000E421D0210F38E421FD308C071930292ABF
:1003A0000C08743E56238C0A08000A148A100A119D
:1003B0000800DB21292A0A148A140A150C08AD004A
:1003C000AD0DAD0D2D070800A003E7297730AA0079
:1003D000AA0932301E227F306600AB018613083036
:1003E000A8001D222A08AB068613AA1B8617AA0D91
:1003F000A80BF1291D228613AB1F86171D22FF3083
:1004000066004F301E2A0422E621861B052A2A3068
:100410001E220930A8000310861F0314AA0D1D22F6
:10042000A80B0B2AAA0C28301E222A0808008523B4
:1004300003106B230318172A08001B30A900A90B0F
:100440001F2A003489008316081483120808080044
:10045000003083170A1463235C23AD00831FE4215B
:10046000A003A01B0D281D1AFF30AD03AD1B3B2AB6
:100470005C23080E963AE721302A3F22402A840066
:100480004322432243220008880009088402080806
:10049000800009088407840A080001300A1A1B300A
:1004A00088000310A4190314A411A70DA60DA50D0F
:1004B000A40DA30DA20DA10D03182416880B512A1B
:1004C00008008800880C080C0800183084000422FA
:1004D0008000840A841E672A0A1E792A1830950033
:1004E00083174523950A951E712A103089002830FC
:1004F0003D221030A0000A1A201E7F2A892A4D2290
:1005000020030319892A0D3C031C892A063A031D7E
:100510004D22D521283094000830970006309600EF
:10052000970A1708222295000739203E8400950D6E
:10053000F03095050318950E150803100005031DEE
:10054000031414088400800D960B902A0013801366
:10055000940A94198E2A9401950197010A101F0C90
:100560001C0C612228063F39562388199517081953
:10057000961788189614081897141D0D1C0D290637
:100580003F394038562388199515081917168818C9
:100590001417081816171C0C1D0C61222A063F3967
:1005A0008038562388191614081915148818171539
:1005B000081814151E0D1D0D2B063F39C038562383
:1005C0008819171708191616881815170818941778
:1005D0001D0C1E0C61222C063F395623881B141457
:1005E000081B1515881A9717081A94161F0D1E0D4B
:1005F0002D063F3940385623881B1416081B9715C3
:10060000881A9516081A96161E0C1F0C61222E06C3
:100610003F3980385623881B1714081B1516881A73
:100620001615081A94141C0D1F0D2F063F39C038DB
:100630005623881B9415081B9716881A9514081AB8
:10064000961518089406190895061A0896061B08A8
:100650009706043089001C303F22F830890014309E
:100660003F22A00B7B2A0A1E00344D221F3095002A
:100670008313452304309506151D392B9503151951
:10068000392B1430890028303D2A2830960015086F
:100690008400831F4E2B800D800D4F2B800C16087D
:1006A0008400800C960A161E472B080089008523BB
:1006B00003106B2309086E23852303146B2379230E
:1006C0008D23080808008900852303106B2309087F
:1006D0006E2B6E238D2B0A0D0F39A0388800CF307A
:1006E000660074237423A92B772377237723880D3F
:1006F0009D2BDF3066007F237F2303149A2B8223F8
:1007000082238223AC23880D08000616CF306600B2
:100710000000861600000612972B0612CF306600E6
:100720000000861600000000061600000000861279
:1007300000000800CF3066000000031C0612000015
:1007400000000318061600000000861600000000D6
:10075000952BDF30660000008616000000000314B1
:0E07600000000000061E031000000000972B92
:08400000FF3FFF3FFF3FFF3FC0
:02400E00F13F80
:104200003F0067002F0000001100140000000300B1
:104210006800A200430012008B004100C1001100A1
:104220000C009200A100C3002200930013000A00BA
:104230000900240089008A00910014000B00C200CC
:10424000210046000F009400C50096009700A400CE
:104250008D001700C60045008E000E004700950037
:104260008F002500C700A600260027000D00C4000F
:104270008C000000000000000000000000000000B2
:00000001FF
